:100000002500000B240CFF0FFF0FFF0FFF0FFF0F4A
:10001000FF0FFF0FFF0FFF0F3000F0067002000808
:1000200020084D084F08440843084808490850086C
:100030002C082008760835082E0836082E083108C6
:10004000200820084308530852082F085208450882
:1000500049082008310839083908390830083308B8
:06006000320837082008F9
:10008000320C2A00A50C2B000400A6070F05EB027A
:10009000440A06072F054C0A4D0A4E0AEA02420A94
:1000A0004F08010C2700480C4109040C28000D02E0
:1000B00077092C006C02080C2900FB0C0600040CCC
:1000C00041092C03F90C26000306FB0C0307F90C6D
:1000D0000600040C4109E902610AF90C0600080C4B
:1000E0004109AD02E802570AE702530A4308E20158
:1000F0005308430845084108530843084508450884
:080100005308430845084908B3
:10020000FF0C060083074E0B820C02006F000209F0
:10021000060C90002E0040090607160B640C270000
:100220002F061B0B4009E702100B4E0B780C270022
:100230004009E702180B40092604FD0C0600100CCB
:1002400027004009E702210B4604F90C060040098B
:100250000606440B060C27004009E7022C0B0E0C87
:10026000410906063F0B6D000F063F0B51090F06B3
:100270003F0B51090F063F0B5109EE02310BEF0CFA
:10028000060040090607410B40090606440B100210
:0E0290002E006F00F90C06004009310B4E0BDA
:021FFE00FE0FD4
:00000001FF
